:10137000434C52544E30310001320000004F6E0099
:101380000000000000010D92041C00000052706D6E
:10139000446D640000010D93041C00000052706D48
:1013A0004D65617300010D97013200000041636BD0
:1013B0004572720000010D9B0436000000537461F9
:1013C0007475730000010D9C040800000154436F04
:1013D0006E76000000010DA00408000001544D6F5E
:1013E000746F720000010DA40406000001494D6FE6
:1013F000746F720000010DA80418000001564D6FB3
:10140000746F720000010DAC0417000001504D6FA5
:10141000746F720000010DB0043600000045727256
:10142000436F646531010DB40436000000457272EB
:10143000436F646532010DB80436000000576172D5
:101440006E436F6465010DBC0436000000496E6692
:101450006F436F6465010DC0013400000864300003
:101460000000000000010DC40134000008643100D8
:101470000000000000010DC50134000008643200C6
:101480000000000000010DC60134000008643300B4
:101490000000000000010DC70134000008643400A2
:1014A0000000000000010DC8013400000864350090
:1014B0000000000000010DC901340000086436007E
:1014C0000000000000010DCA01340000086437006C
:1014D0000000000000010DCB01340000086438005A
:1014E0000000000000010DCC013400000864390048
:1014F0000000000000010DCD01340000086431300F
:101500000000000000010DCE0134000008643131FC
:101510000000000000010DCF0134000008643132EA
:101520000000000000010DD00134000008643133D8
:101530000000000000010DD10134000008643134C6
:101540000000000000010DD20134000008643135B4
:101550000000000000010DD30000000000000000AA
:08156000000000000000000083
:10310000011F01430DD4FF1378440D8E0000000011
:10002600EF600F900D93120EB900000000E4900DE2
:1000360092F0900D9C120EB900000000900DB412C3
:100046000EB900000000900DB8120EB900000000B5
:10005600900DBC120EB900000000900DC0120EB932
:1000660000000000E4FFEFC3941074809480500FEA
:1000760074C42FF582E4340DF583E4F00F80E77D38
:10008600087F01122D8C75840F75A481C287900D8F
:0D0096005A7401F0900D62F0E4FF0232A3F5
:10319C0090FFFF120F40EFF0850883850982E02431
:1031AC0059F582E4340DF5837401F0900001020F9F
:0131BC0040D2
:08000300900DE9EFF07F0022EF
:102ED700900DE9EBF0A3EAF0A3E9F0900DE9E0FB30
:102EE700A3E0FAA3E0F9120CF9FF900DECE0FBA3C5
:102EF700E0FAA3E0F9EF120D3F900DE9E0FBA3E044
:102F0700FAA3E0F9900001120D12FF900DECE0FB1F
:102F1700A3E0FAA3E0F9900001EF120D517F02221E
:102A7100900D7A7403F0A304F0A3EFF0900D7BE0C6
:102A8100FE900D7AE02E2F900D7DF0F404F07B0185
:062A91007A0D797A7D0444
:0E2A9700900DF4EBF0A3EAF0A3E9F0A3EDF04C
:102AA500E4A3F0A3F0900DF7E0FFA3E0FCA3E0FDA5
:102AB500C39FEC94005026900DF4E0FBA3E0FAA32D
:102AC500E0F98D828C83120D12FF122FB7900DF94C
:102AD500E004F070D0900DF8E004F080C81231BD2C
:0B2AE5007A007B327D017F0102236339
:0528EC00900DFAEFF071
:1028F10012325B900DFB120EAD900C0DE0FEA3E0C9
:10290100FF900C15E06E7003A3E06F6028900C0D32
:10291100E475F001120DBF85F082F583E0FF900CA4
:102921000DE0B4080FA3E0B4090A900C0D7400F097
:10293100A37409F02212325BC004C005C006AB07C4
:10294100900DFAE0FFE4FCFDFEA3E0F8A3E0F9A39B
:10295100E0FAA3E02FFFEE3AFEED39FDEC38FCD0B2
:0D29610002D001D000C3120E5C408E7F003A
:01296E002246
:10000E007E007F09900C15EEF0A3EFF0900C0DEE34
:05001E00F0A3EFF02249
:101C6600E4900DF4F0A3F0900DF4E0FEA3E0FFC3C2
:101C76009414EE9400501C74662FF582740D3EF594
:101C860083E4F0900DF5E004F070DC900DF4E004D0
:101C9600F080D47F0A1228EC900D66EFF03395E0C1
:101CA600FE900DF6F0A3EFF04E7003FEFF22D390E8
:101CB6000DF7E09412900DF6E06480948040057E66
:101CC600FF7FFF22900D66E0900DF8F0900DF4E492
:101CD600F0A304F0900DF6E0FEA3E0FFC3900DF52F
:101CE600E09F900DF4E09E503A7F0A1228EC900D8A
:101CF600F4E0FCA3E0FD2466F582740D3CF583EF69
:101D0600F074662DF582740D3CF583E0FF900DF8B6
:101D1600E02FF0900DF5E004F070B9900DF4E004BA
:101D2600F080B1900DF8E0F404F07F0A1228EC90F0
:101D36000DF9EFF0900DF4E0FCA3E02466F5827453
:101D46000D3CF583EFF07A007B327D017F00122394
:101D560063900DF9E0FF900DF8E0B5070A900DF6D7
:0B1D6600E0FEA3E0FF80047EFF7FFF93
:011D7100224F
:10324800900001120D12FE120CF97C002400FFEC14
:033258003EFE2215
:1021F000900DEFEBF0A3EAF0A3E9F0900DEFE0FB18
:10220000A3E0FAA3E0F9900001120D12FFE4FCFD37
:10221000FE7808120E81A804C005C006C007900D04
:10222000EFE0FBA3E0FAA3E0F9120CF9FFD003D032
:1022300002D001EF2BFFE43AFEE439FDE438FCC0A4
:1022400004C005C006C007900DEFE0FBA3E0FAA3B1
:10225000E0F9900002120D12FFE4FCFDFE7810126E
:102260000E81D003D002D001D000EB2FFFEA3EFE5A
:10227000E93DFDE83CFCC004C005C006C007900D68
:10228000EFE0FBA3E0FAA3E0F9900003120D12FFC8
:10229000E4FCFDFE7818120E81D003D002D001D0EC
:0E22A00000EB2FFFEA3EFEE93DFDE83CFC228C
:10296F00E4FFFE900D7A7402F0E4A3F0900D7AE08C
:10297F00900D7CF0F404F07B017A0D797A7D0312CF
:10298F002A97121C66D3EF9400EE64809480405017
:10299F007B017A0D79681221F0900DB4120EAD7B88
:1029AF00017A0D796C1221F0900DB8120EAD7B01EA
:1029BF007A0D79701221F0900DBC120EAD7B017A59
:1029CF000D79741221F0900DC0120EAD900DB8E07C
:1029DF00FCA3E0FDA3E0FEA3E0FF900D9C120EAD63
:0129EF0022C5
:10312A00122A71121C66C3EF940574809480400EB3
:10313A00E4900D9BF07B017A0D7969023248900D7B
:07314A009B7401F0E4FEFF9D
:01315100225B
:1030D600122A71121C66C3EF940774809480400E06
:1030E600E4900D9BF07B017A0D79690221F0900D39
:0930F6009B7401F0E4FFFEFDFCF7
:0130FF0022AE
:10241800900D93E0FCA3E0FDA3E0FEA3E0FF900D88
:06242800F0120EADE4FF0E
:10242E00900D7A7408F0A37405F0A3EFF0A3740373
:10243E00F0900DF0E0FCA3E0FDA3E0FEA3E0FF9022
:10244E000D7EEFF0900DF0A3A3A3E07808120E6DB1
:10245E00900D7FEFF0900DF0E0FCA3E0FDA3E0FE09
:10246E00A3E0FF7810120E6D900D80EFF0900DF03E
:10247E00E0FCA3E0FDA3E0FEA3E0FF7818120E6DD2
:10248E00900D81EFF0E4A3F0FFEFC39408748094F5
:10249E00805015747A2FF582E4340DF583E0FE90AA
:1024AE000D82E02EF00F80E1900D82E0F404F07BBF
:0D24BE00017A0D797A7D09122A97021C66B9
:101D72007E007F147D007B017A0D797A120F717ECD
:101D8200007F147D007B017A0D7966120F71900D30
:101D92007A740AF0A37401F0900DB4E0FCA3E0FDA4
:101DA200A3E0FEA3E0FF900D7CEFF0900DB4A3A39F
:101DB200A3E07808120E6D900D7DEFF0900DB4E067
:101DC200FCA3E0FDA3E0FEA3E0FF7810120E6D90ED
:101DD2000D7EEFF0900DB4E0FCA3E0FDA3E0FEA3C6
:101DE200E0FF7818120E6D900D7FEFF0900DB8E0C5
:101DF200FCA3E0FDA3E0FEA3E0FF900D80EFF090D6
:101E02000DB8A3A3A3E07808120E6D900D81EFF038
:101E1200900DB8E0FCA3E0FDA3E0FEA3E0FF781084
:101E2200120E6D900D82EFF0900DB8E0FCA3E0FD74
:101E3200A3E0FEA3E0FF7818120E6D900D83EFF081
:101E4200E4A3F0FFEFC3940A748094805015747A6F
:101E52002FF582E4340DF583E0FE900D84E02EF040
:101E62000F80E1900D84E0F404F07B017A0D797A21
:081E72007D0B122A97021C6689
:10315200EF900D7A600A7402F0A3F0A374FC800968
:103162007402F0A304F0A374FBF07B017A0D797A68
:083172007D03122A97021C667E
:101E7A00900D59E06017E4F0FA7B327D027F01127F
:101E8A002363122418900D92E0FF123152900D5ADA
:101E9A00E0600FE4F0FA7B327D027F0112236312C5
:101EAA002418900D62E07004A3E06014E4900D62BF
:101EBA00F0A3F0FA7B327D027F01122363121D72B6
:101ECA0012325BA804A905AA06AB07900D8EE0FCA6
:101EDA00A3E0FDA3E0FEA3E02464FFE43EFEE43DAC
:101EEA00FDE43CFCD3120E5C5003021F7A12000E72
:101EFA0012296F7F011230D6900D97120EAD7F0412
:101F0A0012312AAC06AD07EC120C76900DA0120E17
:101F1A00AD7F0812312AAC06AD07EC120C76900D93
:101F2A00A4120EAD7F0212312AAC06AD07EC120CD8
:101F3A0076E4FBFA797A7844120BD4900DA8120E43
:101F4A00AD7F0512312AAC06AD07EC120C76900D66
:101F5A00AC120EAD7F0612312AAC06AD07EC120C9C
:101F6A0076900DB0120EAD12325B900D8E120EAD40
:011F7A002244
:10323300323032322D30372D3132202D203132339E
:053243003435363700B0
:101568007BFF7A3279337D2D122B6FEA494B601F4E
:101578007BFF7A3279337D2D122B6FE92402F9E44F
:101588003AFA900DF3EBF0A3EAF0A3E9F08004E453
:10159800FEFF22900DF3E0FBA3E0FAA3E0F9900030
:1015A80001120D12FF3395E0FEC3EF9430EE648014
:1015B80094804016D3EF9439EE64809480500B9059
:1015C8000001120D1224D0FF802E900001120D127E
:1015D800FF3395E0FEC3EF9461EE6480948040167B
:1015E800D3EF9466EE64809480500B900001120D46
:1015F8001224A9FF80027F00EF7D00FC120CF9FF86
:101608003395E0FEC3EF9430EE64809480401ED39F
:10161800EF9439EE648094805013900DF3E0FBA3AF
:10162800E0FAA3E0F9120CF924D0FF8033900DF30F
:10163800E0FBA3E0FAA3E0F9120CF9FF3395E0FE12
:10164800C3EF9461EE648094804013D3EF9466EE08
:10165800648094805008120CF924A9FF80027F004E
:10166800EFC454F04CFC900DF3E0FBA3E0FAA3E0C8
:10167800F9900002120D12FF3395E0FEC3EF94308B
:10168800EE648094804016D3EF9439EE64809480A1
:10169800500B900002120D1224D0FF8039900DF3E8
:1016A800E0FBA3E0FAA3E0F9900002120D12FF3369
:1016B80095E0FEC3EF9461EE648094804016D3EF0A
:1016C8009466EE64809480500B900002120D1224F0
:1016D800A9FF80027F00EF75F010A4FFE5F04CFE33
:1016E800EF4DFF900DF3E0FBA3E0FAA3E0F99000C3
:1016F80003120D12FD3395E0FCC3ED9430EC6480C9
:1017080094804016D3ED9439EC64809480500B900B
:101718000003120D1224D0FD8039900DF3E0FBA3D5
:10172800E0FAA3E0F9900003120D12FD3395E0FCF6
:10173800C3ED9461EC648094804016D3ED9466EC1C
:1017480064809480500B900003120D1224A9FD8030
:06175800027D00EF4DFFD1
:01175E002268
:10101900E47880F6123281C2B575840F75E104E473
:10102900F5E275E344F58475B7B075840F758A8365
:10103900F597438901758D01758F01758E04900DA2
:10104900F1F0A3F0900DF2E004F07006900DF1E0DC
:1010590004F0900DF1E07004A3E0640F70E6438999
:1010690002E4900DF1F0A3F0900DF1E0FEA3E0FF92
:10107900E4FCFD7B507AC3F9F8D3120E464016E51D
:101089008954107010900DF2E004F070DB900DF1AE
:10109900E004F080D37597021231DCE4FF1231FBD2
:1010A90043EF04E4900DF1F0A3F0900DF1E0FEA3FD
:1010B900E0FFC39402EE940050157D0112303B907D
:1010C9000DF2E004F070E3900DF1E004F080DBE450
:1010D900F520C20AC208C20EC20DC20CD20F788016
:1010E900F608F67826F618F6782CF6900DF1F0A3A6
:1010F900F0900DF1E0FEA3E0FFC3EE9401501C74E3
:10110900192FF582740C3EF583E4F0900DF2E0049A
:10111900F070DE900DF1E004F080D6E4900DF1F06E
:10112900A3F0900DF1E0FEA3E0FFC39440EE94001C
:10113900501C74192FF582740D3EF583E4F0900D5F
:10114900F2E004F070DC900DF1E004F080D412328A
:10115900B4E4F584E5EF54027010E5EF5408D39434
:1011690000748094804003D38001C392037D08E416
:10117900FF122D8CE4782BF67823F6900DD4E0FB42
:10118900A3E0FAA3E0F97823E6FF75F010A4F5824D
:1011990085F083120D12FE782B26F6EE6005782372
:1011A9000680D8D3EF9400748094804035900DD494
:1011B900E0FBA3E0FAA3E0F990000D120EEA120C8D
:1011C900F9FF7455120D3F120CF964556002D20CE7
:1011D90074AA120D3F120CF964AA6002D20CEF1224
:1011E9000D3FE4F584E5EF5402D3940074809480B4
:1011F90040047F018002E4FF1218F2900DF0EFF035
:10120900900DF0E05401703CC20974FF782EF60885
:10121900F608F608F67E007F107D007B007A0079DB
:1012290034120F71900DF674FFF0A37413F0A374C8
:1012390070F0A3E4F0A37410F07B007A0079341203
:101249002CC98002D2091215687832A60608A607A9
:10125900900DF0E054026003021338A3F0A3F0905C
:101269000DF2E0C4F8540FC868FF900DF1E0C454C2
:10127900F048FE900DD4E0FBA3E0FAA3E0F98F82D9
:101289008E83120D12700302132FE92FF9EA3EFA29
:10129900900004120D1220E27CE4900DEFF0900D05
:1012A900EFE0FDC3781F96506C900DF2E0C4F8543E
:1012B9000FC868FF900DF1E0C454F048FE900DD4BA
:1012C900E0FBA3E0FAA3E0F98F828E83120D12FFEF
:1012D9007E00C006C0077C00900DF2E0C4F8540FF0
:1012E900C868FF900DF1E0C454F048FEE92FF9EA0F
:1012F9003EFA90000D120EEA782BE68DF0A429F93A
:10130900EA35F0FA7D00D007D006120F71900DEF83
:10131900E004F08089900DF2E004F07006900DF180
:10132900E004F00212687F01120026C20B8007E474
:10133900FF120026D20BE4900DF1F0A3F0900DF10D
:10134900E0FEA3E0FFC39402EE940050197A007BFB
:10135900967D03122363900DF2E004F070DF900D87
:06136900F1E004F080D762
:01136F00225B
:0532AF00782CE6FF226F
:0632A300EF24FF920F2250
:0632A900A20FE433FF2236
:0300230002175F62
:10175F00C0E0C0F0C083C082C0D075D000C000C050
:10176F0001C002C003C004C005C006C00720990312
:10177F0002180AC2997826067926E7788166703AA8
:04178F00F67826F6CC
:10179300900DD7740AF0900DD7E0D3940074809421
:1017A30080401FA37413F0900DD8E0D3940074808D
:1017B3009480400600E014F080ED900DD7E014F023
:0217C30080D4D0
:0417C500C2B58041E8
:1017C900900DD77414F0900DD7E0D39400748094E1
:1017D90080401FA37413F0900DD8E0D39400748057
:1017E9009480400600E014F080ED900DD7E014F0ED
:0217F90080D49A
:1017FB007826E62419F582E4340DF583E0F599207B
:10180B0098030218D7209A08200A05C2980218D309
:10181B00C29A7825E6062419F582E4340CF583E5A3
:10182B0099F0C298E6FF7E0064017013900C19E0EA
:10183B00FD7004F60218D7ED54072402782DF6EF4D
:10184B0064024E700E782DE664097007900C1AE056
:10185B002403F67825E6FFFD7C00B40007ECB40109
:10186B0003F68068EFC3782D964061ED24FFFDEC05
:10187B0034FFFC7B017A0C79191224CB7825E624F2
:10188B0018F582E4340CF583E06F60047600803C3D
:10189B00900DD77414F0900DD7E0D394007480940E
:1018AB0080401FA37413F0900DD8E0D39400748084
:1018BB009480400600E014F080ED900DD7E014F01A
:0218CB0080D4C7
:1018CD00782A061200A678257600D007D006D00516
:1018DD00D004D003D002D001D000D0D0D082D0839C
:0518ED00D0F0D0E03254
:0532B400782AE6FF226C
:10213000900C1AE075F010A4FF900DD4E0FBA3E022
:10214000FAA3E02FF9EA35F0FA90000D120EEA90AA
:102150000DDB782CE6FF18E68FF0A4FFE02FF58268
:0F216000E435F0F583120D12FF7B017A0D79D96A
:10216F00900DE9EFF0A3EBF0A3EAF0A3E9F0E4F5AB
:10217F0084EA494B6028900DEAE0FBA3E0FAA3E064
:10218F00F9120CF9FF900DE9E0FD7C0012329490EA
:0E219F000DEAE0FBA3E0FAA3E0F9EF120D3F1A
:1021AD00900DED7414F0900DEDE0D39400748094C7
:1021BD0080401FA37413F0900DEEE0D39400748053
:1021CD009480400600E014F080ED900DEDE014F0E9
:0221DD0080D4AC
:1021DF00900DE9E0F5997F011230753099FDC299A4
:0121EF0022CD
:10286200900D197478F07825E62418F582E4340C7A
:09287200F583E0900D1AF07F02DD
:10287B0090FFFF120F40EFF090FFFE120F40E4F5B8
:0F288B0084850883850982A3A3E07881F6D2B5FE
:10289A008508838509827414F0850883850982E096
:1028AA00D3940074809480402DA37413F085088318
:1028BA00850982A3E0D3940074809480400D00853A
:1028CA000883850982A3E014F080E28508838509DC
:0628DA0082E014F080C34F
:0C28E000900D19E0F599900003020F40E4
:102DE000C9EFC9E964017028EDC39B403F781FE635
:102DF000FFEB2FFFE433FEEDC39FEE6480F8748099
:102E0000985029D20AC3ED9B782CF67827760122B8
:102E1000CFE9CFEF6402701ACFEBCFCEEDCEEE6FDD
:102E2000700AD20A782CF67827760222C20AE47851
:032E300027F62260
:10274A00900DE9ECF0A3EDF0C9EFC9BAFF19BBFF90
:10275A0016900DE9E06A7003A3E06B7068D20A78FC
:10276A002CF67827E9F622E964017035C3900DEA60
:10277A00E09B900DE9E09A4026781FE62BFFE43AA9
:10278A00FEE0FCA3E0FDC39FEC9E5013D20ACFEB00
:10279A00CFCEEDCEC3EE9F782CF678277601228035
:1027AA0024CFE9CFEF64027022CEEACECFEBCF90EE
:1027BA000DE9E06E7003A3E06F700AD20A782CF676
:0C27CA007827760222C20AE47827F62263
:1000A600900C19E0FE54F8900DDAF0E4F584EE12A7
:1000B6000F1A00F50901020A011510011E11012F80
:1000C60012014619015C1A018120018A280244297D
:1000D60003AB3303EC37042C39044641045149047D
:1000E6005C5004B06103757004A898000004E090A9
:1000F6000C1AE0FD782FE6FB7F018027900C1AE0B2
:10010600FCA3E0FD782EE6FA08E6FB7F01802BD201
:100116000A782776030204E0900C1AE0FD7831E6AF
:10012600FB7F02122DE00204E0900C1AE0FCA3E033
:10013600FD7830E6FA08E6FB7F0212274A0204E061
:10014600900C1AE0FD782FE6FB7F01122DE0200AC5
:10015600030204E0801A900C1AE0FCA3E0FD782E5E
:10016600E6FA08E6FB7F0112274A200A030204E0AA
:10017600900D197478F07F010204DDE4F58475EFC3
:10018600100204E0C2ACE4900DD9F0D2B57B017A3E
:100196000D79D97F7F12216F7B017A0D79D97F186E
:1001A60012216F7B017A0D79D97F0512216F782391
:1001B600E6122168782EE6122168782FE612216869
:1001C6007830E61221687831E61221687832E61234
:1001D60021687833E6122168E4900DDBF0900DDBA0
:1001E600E0FFC3941074809480501074342FF8E6A6
:1001F600122168900DDBE004F080E2900DD9E0FF5B
:090206007B007A00790012216FDF
:10020F00900DE7740AF0900DE7E0D394007480949A
:10021F0080401FA37413F0900DE8E0D39400748016
:10022F009480400600E014F080ED900DE7E014F0AC
:02023F0080D469
:10024100020360900C1AE0FFC37823964003020377
:1002510067EF75F010A4FF900DD4E0FBA3E0FAA3C3
:10026100E02FF9EA35F0FA900DE4EBF0A3EAF0A300
:10027100E9F0C2ACE4900DD9F0D2B57B017A0D79E9
:10028100D97F7F12216F7B017A0D79D97F0D1221E0
:100291006F900DE4E0FBA3E0FAA3E0F9120CF91270
:1002A1002168900DE4E0FBA3E0FAA3E0F9900001DE
:1002B100122165900DE4E0FBA3E0FAA3E0F99000C0
:1002C10002122165900DE4E0FBA3E0FAA3E0F990AE
:1002D1000003122165900DE4E0FBA3E0FAA3E0F92D
:1002E100900004122165E4900DDBF0900DDBE0FF3E
:1002F100C39408748094805026900DE4E0FBA3E041
:10030100FAA3E02405F9E43AFA7E00E92FF9EE3A7E
:10031100FA120CF9122168900DDBE004F080CC9008
:0D0321000DD9E0FF7B007A00790012216FFA
:10032E00900DE7740AF0900DE7E0D394007480947A
:10033E0080401FA37413F0900DE8E0D394007480F6
:10034E009480400600E014F080ED900DE7E014F08C
:02035E0080D449
:10036000C2B5D2AC0204E0900D197478F0E4A3F0A9
:100370007F020204DD12326E780A120EA1900D196E
:10038000747CF0780AE6A3F008E6A3F008E6A3F090
:1003900008E6A3F07C007D057B017A0D7919122413
:1003A000CB900D1EEFF07F060204DD900C1AE0FFEB
:1003B0007E006401700FA3E0FDA3E0782ECDF60867
:1003C000EDF60204A8EF64024E700A900C1BE07870
:1003D0002EF60204A8900C1AE06403700CA3E0FF50
:1003E000A3E07830CFF608EFF60204A8E4900DDB26
:1003F000F0900DDBE0FFC394107480948050279040
:100400000C1AE0FEEFC39E501D900DDBE0241BF59F
:1004100082E4340CF583E0FE74342FF8EEF6900D90
:10042000DBE004F080CBE47843F6807C7A007B321A
:100430007D01782CE6FF122363900C1AE0FDE4FFA7
:10044000122D8C0204E0900C1AE024FF92020204A8
:10045000E0900C1AE024FF92010204E0782CE660A0
:1004600008900DDD7402F0800E900DDD200D0574F6
:1004700003F080037401F0900D197479F0900DDD94
:10048000E0900D1AF07C007D027B017A0D79191243
:1004900024CB900D1BEFF07F0312287B900DDDE045
:1004A0006401703CD20E8002D208788076F18030F0
:1004B0007A007B327D017F00122363900D197479DD
:1004C000F0900C1AE0900D1AF07C007D027B017A0E
:1004D0000D79191224CB900D1BEFF07F0312287BAE
:1004E000900DDAE064A060030207BF781FE66401A4
:1004F000700D300F0AFA7B327D017F011223639069
:100500000C19E064A16003020650A3E0C3782396AF
:100510004003020645900DD4E0FBA3E0FAA3E0F906
:10052000900C1AE0FF75F010A4F58285F083120D8F
:1005300012900DDDF0EF75F010A4FFE92FF9EA3508
:10054000F0FA900004120D1230E23C900C1AE0FF19
:10055000120003900DDDEFF0900D19747FF0A3EF02
:10056000F02402FDE433FC7B017A0D79191224CBCF
:10057000900DDDE0FE241BF582E4340DF583EFF0F1
:10058000EE2403FF0207BC900C1AE0FF120003C226
:10059000ACE4900DD9F0D2B5900DDDE0D3940674A3
:1005A00080948040377B017A0D79D97F7F12216F4B
:1005B000900DDDE0122168E4900DDBF0900DDDE0A0
:1005C000FF900DDBE0C39F500B122130900DDBE05C
:1005D00004F080E8900DDDE004F08026900DDDE071
:1005E0002478122168E4900DDBF0900DDDE0FF909F
:1005F0000DDBE0C39F500B122130900DDBE004F0C7
:1006000080E8900DD9E0FF7B007A00790012216F1D
:10061000900DE7740AF0900DE7E0D3940074809495
:1006200080401FA37413F0900DE8E0D39400748011
:100630009480400600E014F080ED900DE7E014F0A7
:0206400080D464
:100642000207AE900D197478F07F010207BC900C7E
:1006520019E064A260030207BF7823E6FFA3E0FE6D
:10066200C39F40030207B4A3E0FDC39F40030207F8
:10067200B4EE9D40030207B4900C1AE0900DDBF03B
:10068200E4900DE2F0A3F0900C1BE0FE900DDBE095
:10069200FFD39E5034120003900DD4E0FBA3E0FA86
:1006A200A3E0F9900DDBE075F010A4F58285F083EC
:1006B200120D12FF900DE3E02FF0900DE2E03400F6
:1006C200F0900DDBE004F080BEC2ACE4900DD9F0F6
:1006D200D2B57B017A0D79D97F7F12216F900DE21D
:1006E200E0FEA3E0FFC39480EE94005002800F90DE
:1006F2000DE2E04480122168900DE2A3E0FF122196
:1007020069900C1AE0900DDBF0900C1BE0FF900D4D
:10071200DBE0D39F5056E4A3F0900DD4E0FBA3E0BE
:10072200FAA3E0F9900DDBE0FF75F010A4F58285E5
:10073200F083120D12FE900DDCE0C39E5026EF7581
:10074200F010A4FF900DD4A3A3E02FF9EA35F0FA3C
:1007520090000D120EEA900DDC122152900DDCE099
:1007620004F080B5900DDBE004F0809D900DD9E09F
:0A077200FF7B007A00790012216F6E
:10077C00900DE7740AF0900DE7E0D3940074809428
:10078C0080401FA37413F0900DE8E0D394007480A4
:10079C009480400600E014F080ED900DE7E014F03A
:0207AC0080D4F7
:1007AE00C2B5D2AC800B900D197478F07F0112286F
:1007BE007B900DDAE064587057FA7B327D01782C0D
:1007CE00E6FF122363900DEC7401F0A3740DF0A3F9
:1007DE00741AF07B017A0C791A122ED7900DDDEF78
:1007EE00F0E0FE2478900D19F0EE2401FDE433FCC8
:1007FE007B017A0D79191224CB900DDDE0FE241ABF
:10080E00F582E4340DF583EFF0EE2402FF12287B1F
:10081E00900DDAE0FF64806008EF64886003020ADE
:10082E002C300F367827E66401700EFA7B327D018C
:10083E00782CE6FF1223638021E4900DDBF0900DFF
:10084E00DBE0FFC3781F9650117A007B327D0112D8
:10085E002363900DDBE004F080E4900C19E0540764
:10086E00900DDDF064077012900DDC04F0900C1A00
:10087E00E0900DDDF0900C1B8008E4900DDCF09004
:10088E000C1AE0900DDEF0900DDDE014F0A3E0FF09
:10089E00C37823964003020A2C900DD4E0FBA3E00C
:1008AE00FAA3E0F975F010EFA4F58285F083120D2E
:1008BE0012FF900DDDE0D39F4002EFF07827E66443
:1008CE0001700D782CE6900DE1F0900DE0F0800BAC
:1008DE00E4900DE0F0781FE614A3F0900DE0E078C0
:1008EE002CF6900DE1E0FF782CE6D39F4003020A30
:1008FE001AE4900DDBF0900DDDE0FF900DDBE0C310
:10090E009F4003020A0C900DDEE075F010A4FF90DC
:10091E000DD4E0FBA3E0FAA3E02FF9EA35F0FA904C
:10092E000004120D1230E203020A03900001120DB0
:10093E001264387053900DDDE0D39404748094806B
:10094E00900DDBE0FF4010A3E02F241BF582E43472
:10095E000CF583E0FD807E7825E6C39FFFE49400CE
:10096E00FE74172FF582740C3EF583E0FD900DDEBC
:10097E00E075F010A4FF900DD4E0FBA3E0FAA3E025
:10098E002FF9EA35F0FA804D900DD4E0FBA3E0FA92
:10099E00A3E0F9900DDEE075F010A4F58285F083EA
:1009AE00120D12FF7825E6C39FFFE49400FE900D12
:1009BE00DBE07C002FFFEC3EFE74182FF582740CEA
:1009CE003EF583E0FD900DDEE075F010A4FFE92FFB
:1009DE00F9EA35F0FA90000D120EEA782CE6FF18BF
:1009EE00E68FF0A4FF900DDBE02FF582E435F0F5F5
:1009FE0083ED120D51900DDBE004F0020904900D11
:100A0E00DEE0FF12319C782C060208F0900DE0E03B
:100A1E00782CF6900DDAE064887003122862900D3F
:100A2E00DAE064A86003020BD0300F367827E66454
:100A3E0001700EFA7B327D01782CE6FF1223638063
:100A4E0021E4900DDBF0900DDBE0FFC3781F965094
:100A5E00117A007B327D01122363900DDBE004F0EE
:100A6E0080E4900C1AE030E718547FFEA3E0FDED11
:100A7E00FF900DE2EEF0A3EFF0900DDC7403F0802A
:100A8E0013900C1AE0FF900DE2E4F0A3EFF0900D3E
:100A9E00DC7402F0900DDCE0FF2419F582E4340CD6
:100AAE00F583E0FE741A2FF582E4340CF583E090A2
:100ABE000DDFF0CFEECF900DDEEFF0900DDFE0FF0B
:100ACE00900DDEE0FED39F4003020BCDEEC37823E4
:100ADE00964003020BC4900DD4E0FBA3E0FAA3E012
:100AEE00F975F010EEA4F58285F083120D12900DBB
:100AFE00DDF07827E66401700D782CE6900DE1F0BC
:100B0E00900DE0F0800BE4900DE0F0781FE614A35A
:100B1E00F0900DE0E0782CF6900DE1E0FF782CE6F9
:100B2E00D39F4003020BB2E4900DDBF0900DDDE09D
:100B3E00FF900DDBE0C39F505D900DDEE075F01071
:100B4E00A4FF900DD4E0FBA3E0FAA3E02FF9EA3561
:100B5E00F0FA900004120D1220E233900DDBE0FF4C
:100B6E00A3E02F241BF582E4340CF583E0FD900006
:100B7E000D120EEA782CE6FF18E68FF0A4FF900D0A
:100B8E00DBE02FF582E435F0F583ED120D51900D7B
:100B9E00DBE004F08096900DDEE0FF12319C782CA5
:100BAE0006020B26900DE0E0782CF6900DDDE0FFAE
:100BBE00900DDCE02FF0900DDEE004F0020AC91279
:020BCE0028629B
:010BD0002202
:107000007880E664F16003027B817814F608F678F4
:0470100081E6604372
:10701400900DEF740AF0900DEFE0D3940074809417
:1070240080401FA37413F0900DF0E0D3940074809B
:107034009480400600E014F080ED900DEFE014F031
:0270440080D4F6
:10704600781506E6187001067814B627BC08B6103F
:10705600B8C2AF7584015398FCE47810F618F6E4CC
:10706600F584209855E47814F608F6209848C378F5
:0A70760015E6948818E69413503CC8
:10708000900DEF740AF0900DEFE0D39400748094AB
:1070900080401FA37413F0900DF0E0D3940074802F
:1070A0009480400600E014F080ED900DEFE014F0C5
:0270B00080D48A
:1070B200781506E61870B80680B5B2B480A8780FC5
:1070C200A699C298E6FF641A6008EF640A60030298
:1070D2007267E47814F608F6209848C37815E694A7
:0770E2008818E69413503CEE
:1070E900900DEF740AF0900DEFE0D3940074809442
:1070F90080401FA37413F0900DF0E0D394007480C6
:107109009480400600E014F080ED900DEFE014F05B
:0271190080D420
:10711B00781506E61870B80680B5209803027065DE
:10712B007810A699C298E47814F608F6209848C30C
:0B713B007815E6948818E69413503C89
:10714600900DEF740AF0900DEFE0D39400748094E4
:1071560080401FA37413F0900DF0E0D39400748068
:107166009480400600E014F080ED900DEFE014F0FE
:0271760080D4C3
:10717800781506E61870B80680B520980302706581
:107188007810A699C298E47814F608F6209848C3AF
:0B7198007815E6948818E69413503C2C
:1071A300900DEF740AF0900DEFE0D3940074809487
:1071B30080401FA37413F0900DF0E0D3940074800B
:1071C3009480400600E014F080ED900DEFE014F0A1
:0271D30080D466
:1071D500781506E61870B80680B520980302706524
:1071E5007810A699C29818E6641A6003027B72D2D9
:0371F500B5C29987
:1071F800900DEF7414F0900DEFE0D3940074809428
:1072080080401FA37413F0900DF0E0D394007480B5
:107218009480400600E014F080ED900DEFE014F04B
:0272280080D410
:06722A007599783099FD12
:10723000900DEF740AF0900DEFE0D39400748094F9
:1072400080401FA37413F0900DF0E0D3940074807D
:107250009480400600E014F080ED900DEFE014F013
:0272600080D4D8
:10726200C2B5027B72780FE6FF7E006450600302B3
:1072720073B77814F608F6209848C37815E6948810
:0672820018E69413503CD5
:10728800900DEF740AF0900DEFE0D39400748094A1
:1072980080401FA37413F0900DF0E0D39400748025
:1072A8009480400600E014F080ED900DEFE014F0BB
:0272B80080D480
:1072BA00781506E61870B80680B52098030270653E
:0A72CA007810A699C298D2B5C299B7
:1072D400900DEF7414F0900DEFE0D394007480944B
:1072E40080401FA37413F0900DF0E0D394007480D9
:1072F4009480400600E014F080ED900DEFE014F06F
:0273040080D433
:087306007599793099FDC299D7
:10730E00900DEF7414F0900DEFE0D3940074809410
:10731E0080401FA37413F0900DF0E0D3940074809E
:10732E009480400600E014F080ED900DEFE014F034
:02733E0080D4F9
:087340007599013099FDC29915
:10734800900DEF7414F0900DEFE0D39400748094D6
:1073580080401FA37413F0900DF0E0D39400748064
:107368009480400600E014F080ED900DEFE014F0FA
:0273780080D4BF
:06737A00E4F5993099FDD5
:10738000900DEF740AF0900DEFE0D39400748094A8
:1073900080401FA37413F0900DF0E0D3940074802C
:1073A0009480400600E014F080ED900DEFE014F0C2
:0273B00080D487
:1073B200C2B5027B72EF64014E600302746DD2B5F6
:0273C200C2996E
:1073C400900DEF7414F0900DEFE0D394007480945A
:1073D40080401FA37413F0900DF0E0D394007480E8
:1073E4009480400600E014F080ED900DEFE014F07E
:0273F40080D443
:0873F6007599783099FDC299E8
:1073FE00900DEF7414F0900DEFE0D3940074809420
:10740E0080401FA37413F0900DF0E0D394007480AD
:10741E009480400600E014F080ED900DEFE014F043
:02742E0080D408
:06743000E4F5993099FD1E
:10743600900DEF740AF0900DEFE0D39400748094F1
:1074460080401FA37413F0900DF0E0D39400748075
:107456009480400600E014F080ED900DEFE014F00B
:0274660080D4D0
:10746800C2B5027B72780FE6640260030275CF78BA
:1074780014F608F6209848C37815E6948818E69418
:0374880013503C62
:10748B00900DEF740AF0900DEFE0D394007480949C
:10749B0080401FA37413F0900DF0E0D39400748020
:1074AB009480400600E014F080ED900DEFE014F0B6
:0274BB0080D47B
:1074BD00781506E61870B80680B520980302706539
:1074CD007810A699C298E408F618E6FF13B392B4A3
:1074DD00EF25E0FECC7470CCCD7400CDC3E49DEEF1
:1074ED009C5029E6FD7F0025E0FEC394E0501DED84
:1074FD0020E020E4F58443B701758F037816EEF68E
:10750D0008EFF6F5828E83F0F58F8004781176FF03
:07751D00E4F584D2B5C29928
:10752400900DEF7414F0900DEFE0D39400748094F8
:1075340080401FA37413F0900DF0E0D39400748086
:107544009480400600E014F080ED900DEFE014F01C
:0275540080D4E1
:087556007599783099FDC29986
:10755E00900DEF7414F0900DEFE0D39400748094BE
:10756E0080401FA37413F0900DF0E0D3940074804C
:10757E009480400600E014F080ED900DEFE014F0E2
:02758E0080D4A7
:087590007811E6F5993099FD30
:10759800900DEF740AF0900DEFE0D394007480948E
:1075A80080401FA37413F0900DF0E0D39400748012
:1075B8009480400600E014F080ED900DEFE014F0A8
:0275C80080D46D
:1075CA00C2B5027B72780FE6640360030277DC7847
:1075DA0014F608F6209848C37815E6948818E694B5
:0375EA0013503CFF
:1075ED00900DEF740AF0900DEFE0D3940074809439
:1075FD0080401FA37413F0900DF0E0D394007480BD
:10760D009480400600E014F080ED900DEFE014F052
:02761D0080D417
:10761F00781506E61870B80680B5209803027065D5
:10762F007810A699C298E47814F608F6209848C303
:0B763F007815E6948818E69413503C80
:10764A00900DEF740AF0900DEFE0D39400748094DB
:10765A0080401FA37413F0900DF0E0D3940074805F
:10766A009480400600E014F080ED900DEFE014F0F5
:02767A0080D4BA
:10767C00781506E61870B80680B520980302706578
:10768C007812A699C2987810E6FF1392B4EF25E011
:10769C00FECC7470CCCD7400CDC3E49DEE9C400345
:1076AC00027065E625E0FCC394E04003027065E4DB
:1076BC00F58443B701758F017812E675F020A42488
:1076CC0000FFE5F03C7816F608EFF6E4F584781345
:1076DC00F67813E6C3942074809480503FE408F647
:1076EC0008F6209816C37815E6948818E69413507B
:1076FC000A000806E61870EA0680E7209803027074
:10770C006578160806E618CEE6CE70010614F582EA
:10771C008E83E599F0C29878130680B5E4F584F56C
:07772C008FF584D2B5C2996C
:10773300900DEF7414F0900DEFE0D39400748094E7
:1077430080401FA37413F0900DF0E0D39400748075
:107753009480400600E014F080ED900DEFE014F00B
:0277630080D4D0
:087765007599783099FDC29975
:10776D00900DEF7414F0900DEFE0D39400748094AD
:10777D0080401FA37413F0900DF0E0D3940074803B
:10778D009480400600E014F080ED900DEFE014F0D1
:02779D0080D496
:06779F00E4F5993099FDAC
:1077A500900DEF740AF0900DEFE0D394007480947F
:1077B50080401FA37413F0900DF0E0D39400748003
:1077C5009480400600E014F080ED900DEFE014F099
:0277D50080D45E
:1077D700C2B5027B72780FE6FD7C00640460030289
:1077E700792F7814F608F6209848C37815E6948818
:0677F70018E69413503C5B
:1077FD00900DEF740AF0900DEFE0D3940074809427
:10780D0080401FA37413F0900DF0E0D394007480AA
:10781D009480400600E014F080ED900DEFE014F040
:02782D0080D405
:10782F00781506E61870B80680B5209803027065C3
:10783F007810A699C298E625E07818F608E4F6784D
:10784F0011F67814F608F678180806E618CEE6CE84
:10785F0070010614F5828E83E493781126F678155D
:10786F0006E6187001067815E6700418E6640270D3
:05787F00D6D2B5C2994C
:10788400900DEF7414F0900DEFE0D3940074809495
:1078940080401FA37413F0900DF0E0D39400748023
:1078A4009480400600E014F080ED900DEFE014F0B9
:0278B40080D47E
:0878B6007599783099FDC29923
:1078BE00900DEF7414F0900DEFE0D394007480945B
:1078CE0080401FA37413F0900DF0E0D394007480E9
:1078DE009480400600E014F080ED900DEFE014F07F
:0278EE0080D444
:0878F0007811E6F5993099FDCD
:1078F800900DEF740AF0900DEFE0D394007480942B
:1079080080401FA37413F0900DF0E0D394007480AE
:107918009480400600E014F080ED900DEFE014F044
:0279280080D409
:10792A00C2B5027B72ED64054C6003027B66781473
:10793A00F608F6209848C37815E6948818E6941352
:02794A00503CAF
:10794C00900DEF740AF0900DEFE0D39400748094D6
:10795C0080401FA37413F0900DF0E0D3940074805A
:10796C009480400600E014F080ED900DEFE014F0F0
:02797C0080D4B5
:10797E00781506E61870B80680B520980302706573
:10798E007810A699C298E47814F608F6209848C3A1
:0B799E007815E6948818E69413503C1E
:1079A900900DEF740AF0900DEFE0D3940074809479
:1079B90080401FA37413F0900DF0E0D394007480FD
:1079C9009480400600E014F080ED900DEFE014F093
:0279D90080D458
:1079DB00781506E61870B80680B520980302706516
:0A79EB007812A699C298D2B5C2998D
:1079F500900DEF7414F0900DEFE0D3940074809423
:107A050080401FA37413F0900DF0E0D394007480B0
:107A15009480400600E014F080ED900DEFE014F046
:027A250080D40B
:087A270075997F3099FDC299A9
:107A2F00900DEF7414F0900DEFE0D39400748094E8
:107A3F0080401FA37413F0900DF0E0D39400748076
:107A4F009480400600E014F080ED900DEFE014F00C
:027A5F0080D4D1
:107A61007599203099FD7810E625E0FC7812E675CD
:107A7100F020A42400FFE5F03C7818F608EFF6E4C6
:107A81007811F67813F67813E6C394207480948005
:047A91005061C299E5
:107A9500900DEF7414F0900DEFE0D3940074809482
:107AA50080401FA37413F0900DF0E0D39400748010
:107AB5009480400600E014F080ED900DEFE014F0A6
:027AC50080D46B
:107AC7007818E6FE08E6F5828E83E493F5993099F7
:107AD700FD78180806E618CEE6CE70010614F58282
:0F7AE7008E83E493781126F67813068093C29964
:107AF600900DEF7414F0900DEFE0D3940074809421
:107B060080401FA37413F0900DF0E0D394007480AE
:107B16009480400600E014F080ED900DEFE014F044
:027B260080D409
:087B28007811E6F5993099FD92
:107B3000900DEF740AF0900DEFE0D39400748094F0
:107B400080401FA37413F0900DF0E0D39400748074
:107B50009480400600E014F080ED900DEFE014F00A
:027B600080D4CF
:107B6200C2B5800C780FE664067005F58475EF10D7
:0F7B7200780FE6640760030270657880F6D2AF83
:017B810022E1
:102BE9007F00123075122F7020090B7A007B327D1D
:102BF900017F00122363300C0B7A007B1E7D017F5D
:102C090000122363300817300D147A007B327D01DE
:102C1900782CE6FF122363C208121F7BD209200B0E
:102C29000C300D09788076F1121F7BD20B300E0B18
:102C3900300D08C20E123281127000200D121232AC
:102C49005BE47B2C7A01F9F8C3120E5C5002D20DB9
:012C59002258
:1030AA00E4F58475EF027F64EFD394007480948012
:1030BA0040031F80F31210191232AF12321AE4FFC2
:0C30CA00FE122FFC122BE9121E7A80F877
:101B5200005EBCE2613FDD83C29C7E20A3FD1F418B
:101B62009DC3217FFCA2401E5F01E3BD3E6082DC7B
:101B7200237D9FC1421CFEA0E1BF5D0380DE3C626B
:101B8200BEE0025CDF81633D7C22C09E1D43A1FF5B
:101B92004618FAA427799BC584DA3866E5BB59074B
:101BA200DB856739BAE406581947A5FB7826C49A3B
:101BB200653BD987045AB8E6A7F91B45C6987A242B
:101BC200F8A6441A99C7257B3A6486D85B05E7B91B
:101BD2008CD2306EEDB3510F4E10F2AC2F7193CD0B
:101BE200114FADF3702ECC92D38D6F31B2EC0E50FB
:101BF200AFF1134DCE90722C6D33D18F0C52B0EEEB
:101C0200326C8ED0530DEFB1F0AE4C1291CF2D73DA
:101C1200CA947628ABF517490856B4EA6937D58BCA
:101C22005709EBB536688AD495CB2977F4AA4816BA
:101C3200E9B7550B88D6346A2B7597C94A14F6A8AA
:101C4200742AC896154BA9F7B6E80A54D7896B359A
:101C5200000000002B6096CBDDEE002C96CBDDE57C
:041C6200EEF7FAFDA2
:10311000C191420C0D0009420C150009420C0F0828
:0931200009420C17080901440AD8
:10321A00900DEF120EB9FFFFFFFF900DEFE0FCA338
:08322A00E0FDA3E0FEA3E0FFBC
:013232002279
:1024CB0090FFFE120F40ECF0A3EDF090FFFD120F0A
:0F24DB0040EBF0A3EAF0A3E9F090FFFC120F40F2
:1024EA00850883850982A3A3E4F085088385098288
:1024FA00F0A3F0900007120F64E0FEA3E0FF850846
:10250A0083850982E0FCA3E0FDC39FEE6480F8ECBA
:10251A00648098504C900004120F64E0FBA3E0FA28
:10252A00A3E0F98D828C83120D12FF850883850939
:10253A0082A3A3E06FFF900003120F64EFF09000F4
:10254A0003120F64E0901B5293850883850982A3C6
:10255A00A3F0850883850982E475F001120DA9802C
:0B256A0092850883850982A3A3E0FF8F
:06257500900009020F4076
:0E329400CEEDCEEE6F780EF6E6901B5293FF55
:0132A2002209
:0300A300022AF03E
:102AF000C0E0C0F0C083C082C0D0E8C0E0EEC0E05B
:102B0000EFC0E0E59830E1055398FDD211E598302B
:102B1000E049900C16E02401FF900C15E03400FE13
:102B2000900C0DE06E7003A3E06F7002802A900C91
:102B300015E475F001120DBF85F082F583E599F07B
:102B4000900C15E064087004A3E06409700A900C0E
:102B5000157400F0A37409F05398FED0E0FFD0E0A4
:0F2B6000FED0E0F8D0D0D082D083D0F0D0E032D9
:102F7000900C0FE0FEA3E0FF900C17E06E7003A32F
:102F8000E06F603230112FC211758401900C0FE494
:102F900075F001120DBF85F082F583E0F599900C74
:102FA0000FE0640C7004A3E06409700A900C0F74C5
:072FB00008F0A37409F022F0
:102E3300900C0DE0FEA3E0FF900C15E06E7003A371
:102E4300E06F6039900C0DE475F001120DBF85F051
:102E530082F583E07847F6900C0DE064087004A3D4
:102E6300E06409700A900C0D7400F0A37409F07803
:102E730047E6FEB40D037F0A22CFEECF22122BE9E1
:022E830080AE1F
:062D310090FFFF120F40AD
:102D3700900C0DE0FEA3E0FF900C15E06E7003A36E
:102D4700E06F6039900C0DE475F001120DBF85F04E
:102D570082F583E0850883850982F0900C0DE06495
:102D6700087004A3E06409700A900C0D7400F0A3C6
:0F2D77007409F0850883850982E0FF80027FFFE1
:062D8600900001020F4065
:0E22AE00900E05EBF0A3EAF0A3E9F0A3EDF02B
:1022BC0012325B781A120EA1E4781EF6122D31EF51
:1022CC00FD3395E0FCEDF47002ECF46046EF640A2B
:1022DC006041EFB40D18900E05E0FBA3E0FAA3E00B
:1022EC00F9781EE6FFF582758300E4020D51900E1D
:1022FC0005E0FBA3E0FAA3E0F9781EE606F582758B
:10230C008300EF120D51900E08E0FE781EE6FF6E72
:10231C00700122122BE912325BECC0E0EDC0E0EE52
:10232C00C0E0EFC0E0900E09E0FFE4FCFDFE781A7F
:10233C00120E94EF2BFBEE3AFAED39F9EC38F8D09B
:10234C00E0FFD0E0FED0E0FDD0E0FCD3120E5C400C
:06235C00030222C87F000D
:012362002258
:102FB700900C18E02401FD900C17E03400FC900CF5
:102FC7000FE06C7003A3E06D700122900C17E4759D
:102FD700F001120DBF85F082F583EFF0900C17E03A
:102FE700640C7004A3E06409700A900C177408F06D
:052FF700A37409F022A3
:1031BD00900C0FE0FEA3E0FF900C17E06E7003A3E0
:0F31CD00E06F600A7F00123075122F7080E222CF
:102F27007E007F09900C15EEF0A3EFF0900C0DEEEC
:102F3700F0A3EFF07E087F09900C17EEF0A3EFF0F7
:102F4700900C0FEEF0A3EFF07E087F007D007B0171
:102F57007A007909120F717E047F007D007B017A68
:092F6700087909120F71D2112240
:102D8C00EF7025F5847598D0F584759115F58475DB
:102D9C00C90875CBFFED901C5193F5CA75C804E4B6
:102DAC00F584D2ACC2BC8029758401759850E4F5C9
:102DBC0084E589540F4420F589758E02CFEDCFEF51
:102DCC00901C5B93F58DD28E43E74043F740122F56
:032DDC0027D2AF4C
:012DDF0022D1
:102C5A00900C09120EB900000000900C11120EB966
:102C6A00000000009000007464F0E4780FF6780F1A
:102C7A00E6C39402748094805044E6FF25E025E080
:102C8A002401F582E43400F583E4F0EF25E025E041
:102C9A002402F582E43400F583E4F0EF25E025E030
:102CAA002403F582E43400F583E4F0EF25E025E01F
:0E2CBA002404F582E43400F583E4F00680B0D3
:012CC80022E9
:1031DC00D2AFD2A9C2BBE4F584E589540F4401F502
:0F31EC0089758E02758CAFE4F58AD28C022C5A4D
:061A300090FFFF120F40C1
:101A3600850883850982E4F0850883850982E0FFAD
:101A4600C39402748094804003021B4CEF25E0256A
:101A5600E02404F582E43400F583E0FF7C00D394AF
:101A660000748094805003021B17850883850982C1
:101A7600E025E025E02402F582E43400F583E06009
:101A860003021B17EF30E00DD3940174809480405D
:101A9600047D0080027D01850883850982E0FF12AE
:101AA600257B850883850982E0FF25E025E024045F
:101AB600F582E43400F583E0640170057D011225AA
:101AC6007B850883850982E0FF25E025E02404F56F
:101AD60082E43400F583E014F0EF25E025E02404E9
:101AE600F582E43400F583E0602785088385098262
:101AF600E0FF25E025E02403F582E43400F583E0E9
:101B0600FEEF25E025E02402F582E43400F583EEBD
:101B1600F0850883850982E0FF25E025E02402F5AB
:101B260082E43400F583E06011EF25E025E024022D
:101B3600F582E43400F583E014F085088385098294
:061B4600E004F0021A3E6B
:061B4C00900001020F40B1
:03000B00022619B1
:10261900C0E0C0F0C083C082C0D0E8C0E0E9C0E03B
:10262900EAC0E0EBC0E0ECC0E0EDC0E0EEC0E0EFF6
:10263900C0E0758CAF900C09E0FCA3E0FDA3E0FEBF
:10264900A3E02401FFE43EFEE43DFDE43CFC900CE4
:1026590009120EAD900000E014F0E07025900C1105
:10266900E0FCA3E0FDA3E0FEA3E02401FFE43EFEBD
:10267900E43DFDE43CFC900C11120EAD9000007499
:1026890064F0121A3012317AD0E0FFD0E0FED0E0C7
:10269900FDD0E0FCD0E0FBD0E0FAD0E0F9D0E0F8E2
:0B26A900D0D0D082D083D0F0D0E0323F
:10303B0090FFFF120F40EDF090FFFF120F40EFF0EB
:10304B00850883850982E0FFC394027480948050C5
:10305B0013A3E0FEEF25E025E02401F582E4340024
:0A306B00F583EEF0900002020F4022
:1023630090FFFE120F40EAF0A3EBF090FFFF120F75
:1023730040EDF090FFFF120F40EFF08508838509D1
:1023830082E0FFC39402748094804003022412EF1E
:1023930025E025E02404F582E43400F583E0706F42
:1023A300850883850982E0FB25E025E02402F58288
:1023B300E43400F583E07057850883850982A3E040
:1023C30025E004FF850883850982E0FA25E025E0FE
:1023D3002404F582E43400F583EFF085088385094E
:1023E30082A3A3E0FEA3E0FF7C007D0A120D73EA43
:1023F30025E025E02403F582E43400F583EFF0EBD8
:1024030025E025E02402F582E43400F583E4F0902E
:052413000004020F406F
:10257B0090FFFF120F40EDF090FFFF120F40EFF0B6
:06258B0090FFFF120F405B
:10259100850883850982A3E0FFFD7C00C394027452
:1025A100809480502CEF25E025E02401F582E4346D
:1025B10000F583E0601B850883850982A3A3E07091
:1025C100047F0180027F00850883850982A3A3EF30
:1025D100F0850883850982E584F075840FED4C70E0
:1025E1000F850883850982A3A3E024FF92B4801993
:1025F100850883850982A3E06401700D85088385C0
:102601000982A3A3E024FF92B3850883850982E0B0
:02261100F5844E
:06261300900003020F40DD
:10325B00C2AF900C09E0FCA3E0FDA3E0FEA3E0FFEE
:02326B00D2AFE0
:01326D00223E
:10326E00C2AF900C11E0FCA3E0FDA3E0FEA3E0FFD3
:02327E00D2AFCD
:01328000222B
:1030750090FFFF120F40EFF0850883850982E0700D
:10308500057845F608F63010167844E675F064A420
:10309500FFC37846E69F18E695F0500375FFA590A7
:0530A5000001020F40D4
:1031FB00D210E47845F608F6EF78446003F68002C7
:0F320B00760A75FF0775FFA5E4F58475EF0422B9
:10328100C210E47845F608F6784476FF75FFDE75DE
:03329100FFAD226C
:10317A00784606E6187001063010167844E675F0AF
:10318A0064A4FFC37846E69F18E695F0500375FFDE
:02319A00A5226C
:082FFC00900DEFEEF0A3EFF0E1
:10300400E4A3F0A3F0900DEFE0FEA3E0FFC3900D66
:10301400F2E09F900DF1E09E501C7FE87E031229A0
:10302400F07F01123075900DF2E004F070D7900D2E
:06303400F1E004F080CF82
:01303A002273
:0829F000900DF3EEF0A3EFF0EF
:1029F800D394FAEE94005023900DF3A3E0FFEFD3A5
:102A080094007480948040607E16EED394007480A5
:102A180094804004001E80F21F80E3900DF3E0FFD5
:102A2800A3E0A3CFF0A3EFF0D3900DF6E094FA90D3
:102A38000DF5E0940040177FFA7E001229F0900D02
:102A4800F6E02406F0900DF5E034FFF080DAD3903C
:102A58000DF4E09400900DF3E09400400B900DF518
:082A6800E0FEA3E0FF1229F0DB
:012A70002243
:1026B400900DFF7401F0A3740DF0A374F9F07B0185
:0626C4007A0D79F77D029A
:0E26CA00900DFBEBF0A3EAF0A3E9F0A3EDF016
:1026D8007F01123075900DFFE0FBA3E0FAA3E0F94B
:1026E800120DD52400FFE5F034E0FE900DFBE0F973
:1026F800A3E0FAA3E0900E02C9F0A3EAF0A3E9F080
:10270800E4FD900DFEE0FCEDC39C5022EF2DF58218
:10271800E43EF583E493FC900E02E0FBA3E0FAA309
:10272800E0F98D82758300EC120D510D80D4900D67
:10273800FEE0FFA3E0FBA3E0FAA3E0F9E48FF002D8
:022748000E0081
:10205800900DF17412F0A37434F0900DF97401F03E
:10206800A3740DF0A374F3F07B017A0D79F17D026E
:0E207800900DF5EBF0A3EAF0A3E9F0A3EDF074
:102086007880E664F1600302212F123281C2AFE448
:10209600F58443B701758F01A3E0FBA3E0FAA3E043
:1020A600F9120DD52400FFE5F034E0780FF608EFBD
:1020B600F6900DF5E0FBA3E0FAA3E0F97813C6EB82
:1020C600C608C6EAC608C6E9C6E47811F6900DF851
:1020D600E0FF7811E6C39F50327813CBE6CB0808B1
:1020E60006E618CAE6CA70010614F9120CF9781247
:1020F600F6E6FF780F0806E618CCE6CC7001061463
:10210600F5828C83EFF078110680C2E4F58F900D8E
:10211600F8E0FFA3E0FBA3E0FAA3E0F9E48FF012F6
:092126000E00D2AFE4FF1231FB00
:01212F00228D
:102E85007880E664F1704AC2AF123281E4F584437A
:102E9500B701758F03781076E008F6780FF6780F8E
:102EA500E6C3940874809480501E08E6FE08E6F593
:102EB500828E83E4F07F011230757811E426F618CE
:102EC500740236F6180680D6E4F58FD2AFFF1231BC
:012ED500FB01
:012ED60022D9
:101F7B00122E85E4900DF3F0A3F07B01900DF90484
:101F8B00F0A3740DF0A374F3F01B7A00792E7D1679
:101F9B00122078122058E4900DF0F0900DF0E0C371
:101FAB00781F964003022050E4900DEFF0900DD473
:101FBB00E0FBA3E0FAA3E0F9900DEFE0FF75F01062
:101FCB00A4F58285F083120D126071EF75F010A4E9
:101FDB00FF900DD4A3A3E02FF9EA35F0FA90000D92
:101FEB00120EEA900DF0E0FF782BE68FF0A429F9A2
:101FFB00EA35F0FAEBC0E0EAC0E0E9C0E0900DD4BE
:10200B00E0FBA3E0FAA3E0F9900DEFE075F010A46C
:10201B00F58285F083120D12FD900DF97401F0A37A
:10202B00740DF0A374F3F0D0E0F9D0E0FAD0E0FB3C
:10203B00122078900DEFE004F0021FB8900DF0E045
:0C204B0004F0021FA6122058E47880F672
:012057002266
:0518F200900DF3EFF082
:1018F700E4900DF9F0A3F0900DF6F07B01900DFF49
:1019070004F0A3740DF0A374F9F01B7A00792E7D0F
:10191700161226CA1226B4900DF7E0B4120CA3E0F3
:10192700B43407900DF6E04401F0E4900DF5F09023
:101937000DF5E0C3781F964003021A14E4900DF4E6
:10194700F0900DD4E0FBA3E0FAA3E0F9900DF4E0EA
:10195700FF75F010A4F58285F083120D1270030253
:101967001A0B900DF3E0606AEF75F010A4FF900D6D
:10197700D4A3A3E02FF9EA35F0FA90000D120EEA8E
:10198700900DF5E0FF782BE68FF0A429F9EA35F002
:10199700FAEBC0E0EAC0E0E9C0E0900DD4E0FBA3B9
:1019A700E0FAA3E0F9900DF4E075F010A4F5828554
:1019B700F083120D12FD900DFF7401F0A3740DF06A
:1019C700A374F9F0D0E0F9D0E0FAD0E0FB1226CA10
:1019D7008029900DD4E0FBA3E0FAA3E0F9900DF481
:1019E700E075F010A4F58285F083120D12FF900DBB
:1019F700FAE02FF0900DF9E03400F0900DF4E004D8
:101A0700F0021948900DF5E004F00219361226B4D9
:101A1700900DF7E0B4120CA3E0B43407900DF6E094
:081A27004402F0900DF6E0FF0F
:011A2F002294
:100BD100020CEEEC5D046005E859047003020CE4BC
:100BE100120CAF580460F6EC4860F2EC7004FDFEA4
:100BF100FF22C860DB2481C85009C39860025006F7
:100C0100020CEB9850CAF582E9294B4A7005AB8278
:100C1100020CDA75F0007C1A7880C3EF9BEE9AED36
:100C210099400DC3EF9BFFEE9AFEED99FDE842F06E
:100C3100DC23ACF0D0E0FFD0E0FED0E0FDAB8220C1
:100C4100E7101BEB60BAEC2CFCEF33FFEE33FEED4B
:100C510033FD020CC6E803F830E705C0F075F0007B
:100C6100EF2FFFEE33FEED33FD40B830E7C280AA2F
:100C710075F020800E75F010800575F0087D007EFE
:100C8100007F003392D530D503120E38EC3340107B
:100C9100EF33FFEE33FEED33FDEC33FCD5F0ED2207
:0E0CA100E5F0247EA2D513CC92E7CDCEFF2243
:100CAF00E9D2E7C933E833F892D5EDD2E7CD33EC8B
:070CBF0033FC5002B2D52204
:100CC600EC30E7100FBF000C0EBE00080DBD00048F
:100CD6000BEB6014A2D5EB13FCED92E7FD2274FF3B
:100CE600FCFDFEFF22E480F8A2D574FF13FC7D8094
:030CF600E480EFA8
:030000000227D6FE
:0C27D600787FE4F6D8FD75818102281D93
:100CF900BB010689828A83E0225002E722BBFE02F9
:090D0900E32289828A83E493222B
:100D1200BB010CE58229F582E5833AF583E0225096
:100D220006E92582F8E622BBFE06E92582F8E222E0
:0D0D3200E58229F582E5833AF583E49322FA
:100D3F00BB010689828A83F0225002F722BBFE0193
:020D4F00F3228D
:100D5100F8BB010DE58229F582E5833AF583E8F0D8
:100D6100225006E92582C8F622BBFE05E92582C884
:020D7100F2226C
:100D7300C2D5EC30E709B2D5E4C39DFDE49CFCEE9B
:100D830030E715B2D5E4C39FFFE49EFE120F9DC367
:100D9300E49DFDE49CFC8003120F9D30D507C3E462
:060DA3009FFFE49EFE220A
:100DA900C5F0F8A3E028F0C5F0F8E58215827002D5
:060DB9001583E038F02272
:100DBF00A3F8E0C5F025F0F0E582158270021583E7
:060DCF00E0C838F0E82244
:100DD500BB010A89828A83E0F5F0A3E022500687E9
:100DE500F009E71922BBFE07E3F5F009E3192289AB
:0B0DF500828A83E493F5F074019322DE
:100E0000BB010789828A83020DA9500B09C5F0270F
:100E1000F7C5F01937F722BBFE0D09F8E325F0F30B
:100E2000C5F019E338F322F889828A837401932587
:080E3000F0C5F0F8E49338224C
:0E0E3800C3E49FFFE49EFEE49DFDE49CFC22CB
:100E4600EB9FF5F0EA9E42F0E99D42F0EC6480C823
:060E560064809845F022C3
:100E5C00EB9FF5F0EA9E42F0E99D42F0E89C45F0EC
:010E6C002263
:100E6D00E86010ECA2E713FCED13FDEE13FEEF139B
:040E7D00FFD8F02288
:100E8100E8600FEFC333FFEE33FEED33FDEC33FCCF
:030E9100D8F12273
:0D0E9400E6FB08E6F908E6FA08E6CBF822CE
:0C0EA100ECF608EDF608EEF608EFF6227D
:0C0EAD00ECF0A3EDF0A3EEF0A3EFF022B8
:100EB900A8828583F0D083D082120ED0120ED01270
:100EC9000ED0120ED0E473E493A3C583C5F0C58395
:100ED900C8C582C8F0A3C583C5F0C583C8C582C883
:010EE90022E6
:100EEA00BB010DE58229F582E5833AF583020FFB02
:100EFA005007E92582F8020FF2BBFE07E92582F8BE
:100F0A00021004E58229F582E5833AF58302100D81
:100F1A00D083D082F8E4937012740193700DA3A366
:100F2A0093F8740193F5828883E47374029368607A
:060F3A00EFA3A3A380DF7A
:100F4000E5092582F582E5083583F583B508048532
:100F500082092210AF06858209F50822858209F5EB
:040F600008D2AF22E2
:0D0F6400E5092582F582E5083583F5832235
:102CC900900DF3EBF0A3EAF0A3E9F0E4900DFBF02B
:102CD900A3F0900DF974FFF5F0120DBF45F0603CBB
:102CE900900DF6E0FBA3E0FAA3E0F9120CF9FF90CE
:102CF9000DF3E0FBA3E0FAA3E0F9900DFBE475F016
:102D090001120DBF85F082F583EF120D51EF60C2FC
:102D1900900DF7E475F001120DA980B6900DF3E05E
:082D2900FBA3E0FAA3E0F9228C
:102B6F00900DF6EBF0A3EAF0A3E9F0A3EBF0A3EAE4
:102B7F00F0A3E9F0900DF9E0FBA3E0FAA3E0F9125E
:102B8F000CF9600C900DFAE475F001120DA980E4B8
:102B9F00900DF9E0FBA3E0FAA3E0F9120CF96D70C8
:102BAF000122900DF6E0FBA3E0FAA3E0F9EBC0E001
:102BBF00EAC0E0E9C0E0A3E0FBA374FFF5F0120D5B
:102BCF00BFFAD082D083D0E06B7009E5F0658270D8
:0A2BDF0003EA658370BAFBFAF922DD
:100F7100EF4E6012EF60010EEDBB010B89828A8397
:100F8100F0A3DFFCDEFA2289F05007F709DFFCA9A4
:0C0F9100F022BBFEFCF309DFFCA9F022FB
:1027E2000230AAE493A3F8E493A34003F68001F233
:1027F20008DFF48029E493A3F85407240CC8C333F8
:10280200C4540F4420C8834004F456800146F6DFC6
:10281200E4800B0102040810204080903100E47E25
:10282200019360BCA3FF543F30E509541FFEE493BB
:10283200A360010ECF54C025E060A840B8E493A382
:10284200FAE493A3F8E493A3C8C582C8CAC583CAAD
:10285200F0A3C8C582C8CAC583CADFE9DEE780BE65
:0131290000A5
:100F9D00BC000BBE0029EF8DF084FFADF022E4CC38
:100FAD00F875F008EF2FFFEE33FEEC33FCEE9DEC01
:100FBD00984005FCEE9DFE0FD5F0E9E4CEFD22ED47
:100FCD00F8F5F0EE8420D21CFEADF075F008EF2F91
:100FDD00FFED33FD4007985006D5F0F222C398FD82
:050FED000FD5F0EA221F
:090FF200E6FB08E6FA08E6F92224
:090FFB00E0FBA3E0FAA3E0F922F7
:09100400E2FB08E2FA08E2F9221D
:0C100D00E493FB740193FA740293F9223F
:00000001FF
